 BUSPCIE950

 Timestamp is 49d37343 (Wed Apr 01 14:59:31 2009)

 Preferred load address is 10000000

 Start         Length     Name                   Class
 0001:00000000 000009d0H .rdata                  CODE
 0001:000009d0 00000027H .rdata$debug            CODE
 0001:000009f8 0000249cH .text                   CODE
 0001:00002e94 00000028H .idata$2                CODE
 0001:00002ebc 00000014H .idata$3                CODE
 0001:00002ed0 00000098H .idata$4                CODE
 0001:00002f68 00000016H .idata$6                CODE
 0001:00002f80 00000057H .edata                  CODE
 0002:00000000 00000098H .idata$5                DATA
 0002:00000098 0000044cH .data                   DATA
 0002:000004e8 0000010cH .bss                    DATA

  Address         Publics by Value              Rva+Base       Lib:Object

 0000:00000000       ___safe_se_handler_table   00000000     <absolute>
 0000:00000000       ___safe_se_handler_count   00000000     <absolute>
 0001:0000001c       ??_C@_1BI@IGMEDLLH@?$AA?$CF?$AAs?$AA?2?$AAU?$AAn?$AAi?$AAm?$AAo?$AAd?$AAe?$AAm?$AA?$AA@ 1000101c     buspcie950.obj
 0001:00000034       ??_C@_1BK@BFIEKNFP@?$AAF?$AAr?$AAi?$AAe?$AAn?$AAd?$AAl?$AAy?$AAN?$AAa?$AAm?$AAe?$AA?$AA@ 10001034     buspcie950.obj
 0001:00000050       ??_C@_19OBNDINH@?$AAP?$AAo?$AAr?$AAt?$AA?$AA@ 10001050     buspcie950.obj
 0001:0000005c       ??_C@_1BG@KCOOGCNN@?$AAD?$AAe?$AAv?$AAi?$AAc?$AAe?$AAT?$AAy?$AAp?$AAe?$AA?$AA@ 1000105c     buspcie950.obj
 0001:00000074       ??_C@_1BK@HFHDBJKI@?$AAU?$AAn?$AAi?$AAm?$AAo?$AAd?$AAe?$AAm?$AA?4?$AAd?$AAl?$AAl?$AA?$AA@ 10001074     buspcie950.obj
 0001:00000090       ??_C@_1BO@DLFIJDKP@?$AA?$CF?$AAs?$AA?2?$AAS?$AAe?$AAr?$AAi?$AAa?$AAl?$AAC?$AAa?$AAb?$AAl?$AAe?$AA?$AA@ 10001090     buspcie950.obj
 0001:000000b0       ??_C@_15GANGMFKL@?$AA?$CF?$AAs?$AA?$AA@ 100010b0     buspcie950.obj
 0001:000000b8       ??_C@_11LOCGONAA@?$AA?$AA@ 100010b8     buspcie950.obj
 0001:000000bc       ??_C@_1CA@INOAHGHF@?$AAB?$AAu?$AAs?$AAA?$AAc?$AAc?$AAe?$AAs?$AAs?$AAH?$AAa?$AAn?$AAd?$AAl?$AAe?$AA?$AA@ 100010bc     buspcie950.obj
 0001:000000dc       ??_C@_1O@GBAEOCCH@?$AAP?$AAr?$AAe?$AAf?$AAi?$AAx?$AA?$AA@ 100010dc     buspcie950.obj
 0001:000000ec       ??_C@_1BE@GPBAGNPC@?$AAI?$AAs?$AAr?$AAH?$AAa?$AAn?$AAd?$AAl?$AAe?$AA?$AA@ 100010ec     buspcie950.obj
 0001:00000100       ??_C@_1BC@MCDIKBIL@?$AAI?$AAs?$AAt?$AAE?$AAv?$AAe?$AAn?$AAt?$AA?$AA@ 10001100     buspcie950.obj
 0001:00000114       ??_C@_1BG@LJAMCNJN@?$AAP?$AAo?$AAr?$AAt?$AAN?$AAu?$AAm?$AAb?$AAe?$AAr?$AA?$AA@ 10001114     buspcie950.obj
 0001:0000012c       ??_C@_1CC@KMPFMANC@?$AAD?$AAe?$AAv?$AAi?$AAc?$AAe?$AAA?$AAr?$AAr?$AAa?$AAy?$AAI?$AAn?$AAd?$AAe?$AAx?$AA?$AA@ 1000112c     buspcie950.obj
 0001:00000150       ??_C@_17DJMMGLBL@?$AAD?$AAl?$AAl?$AA?$AA@ 10001150     buspcie950.obj
 0001:00000158       ??_C@_17KKLPNNMB@?$AAC?$AAO?$AAM?$AA?$AA@ 10001158     buspcie950.obj
 0001:00000160       ??_C@_1BE@EODMIMC@?$AA?$CF?$AAs?$AA?2?$AAp?$AAo?$AAr?$AAt?$AA?$CF?$AAd?$AA?$AA@ 10001160     buspcie950.obj
 0001:00000174       ??_C@_1CM@HIMBKDJM@?$AAL?$AAi?$AAn?$AAe?$AAD?$AAr?$AAi?$AAv?$AAe?$AAr?$AAD?$AAe?$AAl?$AAa?$AAy?$AAP?$AAh?$AAa?$AAs?$AAe?$AAs?$AA?$AA@ 10001174     buspcie950.obj
 0001:000001a0       ??_C@_1CI@GLAIJPLJ@?$AAL?$AAi?$AAn?$AAe?$AAD?$AAr?$AAi?$AAv?$AAe?$AAr?$AAD?$AAe?$AAl?$AAa?$AAy?$AAB?$AAi?$AAt?$AAs?$AA?$AA@ 100011a0     buspcie950.obj
 0001:000001c8       ??_C@_1CI@OJPKJBA@?$AAB?$AAa?$AAu?$AAd?$AAr?$AAa?$AAt?$AAe?$AAM?$AAa?$AAp?$AAL?$AAi?$AAs?$AAt?$AAF?$AAr?$AAo?$AAm?$AA?$AA@ 100011c8     buspcie950.obj
 0001:000001f0       ??_C@_1CE@BHEKDMEI@?$AAB?$AAa?$AAu?$AAd?$AAr?$AAa?$AAt?$AAe?$AAM?$AAa?$AAp?$AAL?$AAi?$AAs?$AAt?$AAT?$AAo?$AA?$AA@ 100011f0     buspcie950.obj
 0001:00000214       ??_C@_1BE@DDEHHBPD@?$AAD?$AAe?$AAv?$AAC?$AAo?$AAn?$AAf?$AAi?$AAg?$AA?$AA@ 10001214     buspcie950.obj
 0001:00000228       ??_C@_17KNDIACFJ@?$AAT?$AAs?$AAp?$AA?$AA@ 10001228     buspcie950.obj
 0001:00000230       ??_C@_1BG@JDAFHBOG@?$AAI?$AAS?$AAR?$AAH?$AAa?$AAn?$AAd?$AAl?$AAe?$AAr?$AA?$AA@ 10001230     buspcie950.obj
 0001:00000248       ??_C@_1BG@NELPJJNN@?$AAI?$AAs?$AAr?$AAH?$AAa?$AAn?$AAd?$AAl?$AAe?$AAr?$AA?$AA@ 10001248     buspcie950.obj
 0001:00000260       ??_C@_1BO@KACPNJCM@?$AAi?$AAs?$AAr?$AAp?$AAc?$AAi?$AAe?$AA9?$AA5?$AA0?$AA?4?$AAd?$AAl?$AAl?$AA?$AA@ 10001260     buspcie950.obj
 0001:00000280       ??_C@_1O@MDNCMDKF@?$AAI?$AAs?$AAr?$AAD?$AAl?$AAl?$AA?$AA@ 10001280     buspcie950.obj
 0001:00000290       ??_C@_1BO@NHAHMBJD@?$AAc?$AAo?$AAm?$AAp?$AAc?$AAi?$AAe?$AA9?$AA5?$AA0?$AA?4?$AAd?$AAl?$AAl?$AA?$AA@ 10001290     buspcie950.obj
 0001:000002b0       ??_C@_1BA@CEFELOID@?$AAU?$AAa?$AAr?$AAt?$AAD?$AAl?$AAl?$AA?$AA@ 100012b0     buspcie950.obj
 0001:000002c0       ??_C@_1BA@BDHDGOBO@?$AAS?$AAy?$AAs?$AAI?$AAn?$AAt?$AAr?$AA?$AA@ 100012c0     buspcie950.obj
 0001:000002d0       ??_C@_17DJGGJCGD@?$AAI?$AAr?$AAq?$AA?$AA@ 100012d0     buspcie950.obj
 0001:000002d8       ??_C@_1BM@MHMIAMLB@?$AAI?$AAn?$AAt?$AAe?$AAr?$AAf?$AAa?$AAc?$AAe?$AAT?$AAy?$AAp?$AAe?$AA?$AA@ 100012d8     buspcie950.obj
 0001:000002f4       ??_C@_1BE@MNDDMKMB@?$AAB?$AAu?$AAs?$AAN?$AAu?$AAm?$AAb?$AAe?$AAr?$AA?$AA@ 100012f4     buspcie950.obj
 0001:00000308       ??_C@_1O@LBBNFMDB@?$AAM?$AAe?$AAm?$AAL?$AAe?$AAn?$AA?$AA@ 10001308     buspcie950.obj
 0001:00000318       ??_C@_1BA@INLDIDEN@?$AAM?$AAe?$AAm?$AAB?$AAa?$AAs?$AAe?$AA?$AA@ 10001318     buspcie950.obj
 0001:00000328       ??_C@_1M@PEPOCCHH@?$AAI?$AAo?$AAL?$AAe?$AAn?$AA?$AA@ 10001328     buspcie950.obj
 0001:00000334       ??_C@_1O@JMCNHCBG@?$AAI?$AAo?$AAB?$AAa?$AAs?$AAe?$AA?$AA@ 10001334     buspcie950.obj
 0001:00000344       ??_C@_1CE@PJBMNJAF@?$AAL?$AAi?$AAn?$AAe?$AAD?$AAr?$AAi?$AAv?$AAe?$AAr?$AAC?$AAo?$AAn?$AAt?$AAr?$AAo?$AAl?$AA?$AA@ 10001344     buspcie950.obj
 0001:00000368       ??_C@_1CE@HLGCKFJ@?$AAF?$AAl?$AAo?$AAw?$AAC?$AAt?$AAr?$AAl?$AAH?$AAi?$AAg?$AAh?$AAL?$AAe?$AAv?$AAe?$AAl?$AA?$AA@ 10001368     buspcie950.obj
 0001:0000038c       ??_C@_1CC@ELLFOF@?$AAF?$AAl?$AAo?$AAw?$AAC?$AAt?$AAr?$AAl?$AAL?$AAo?$AAw?$AAL?$AAe?$AAv?$AAe?$AAl?$AA?$AA@ 1000138c     buspcie950.obj
 0001:000003b0       ??_C@_1BO@MCGADMLE@?$AAR?$AAx?$AAI?$AAn?$AAt?$AAT?$AAr?$AAi?$AAg?$AAL?$AAe?$AAv?$AAe?$AAl?$AA?$AA@ 100013b0     buspcie950.obj
 0001:000003d0       ??_C@_1BO@ELCCHGIE@?$AAT?$AAx?$AAI?$AAn?$AAt?$AAT?$AAr?$AAi?$AAg?$AAL?$AAe?$AAv?$AAe?$AAl?$AA?$AA@ 100013d0     buspcie950.obj
 0001:000003f0       ??_C@_1CC@EKOCNIBB@?$AAC?$AAr?$AAy?$AAs?$AAt?$AAa?$AAl?$AAF?$AAr?$AAe?$AAq?$AAu?$AAe?$AAn?$AAc?$AAy?$AA?$AA@ 100013f0     buspcie950.obj
 0001:00000414       ??_C@_1BK@KAMHHDIE@?$AAB?$AAr?$AAa?$AAn?$AAd?$AAi?$AAn?$AAg?$AAF?$AAi?$AAl?$AAe?$AA?$AA@ 10001414     buspcie950.obj
 0001:00000430       ??_C@_1BM@CMGCPMHF@?$AAR?$AAe?$AAa?$AAd?$AAB?$AAr?$AAa?$AAn?$AAd?$AAF?$AAi?$AAl?$AAe?$AA?$AA@ 10001430     buspcie950.obj
 0001:0000044c       ??_C@_17KACEIPNC@?$AAK?$AAe?$AAy?$AA?$AA@ 1000144c     buspcie950.obj
 0001:00000454       ??_C@_1DK@IPGGKJ@?$AAH?$AAa?$AAy?$AAe?$AAs?$AA?5?$AAC?$AAo?$AAm?$AAp?$AAa?$AAt?$AAi?$AAb?$AAl?$AAe?$AA?5?$AAo?$AAn?$AA?5?$AAC?$AAO?$AAM?$AA?5?$AAP?$AAo?$AAr?$AAt?$AA?$AA@ 10001454     buspcie950.obj
 0001:00000490       ??_C@_1DC@JFNGNCBP@?$AAS?$AAe?$AAr?$AAi?$AAa?$AAl?$AA?5?$AAC?$AAa?$AAb?$AAl?$AAe?$AA?5?$AAo?$AAn?$AA?5?$AAC?$AAO?$AAM?$AA?5?$AAP?$AAo?$AAr?$AAt?$AA?$AA@ 10001490     buspcie950.obj
 0001:000004c4       ??_C@_1M@FFLAJJMG@?$AA?$DM?$AAE?$AAN?$AAD?$AA?$DO?$AA?$AA@ 100014c4     ConfigParser.obj
 0001:000004d0       ??_C@_1CG@LGKPGFHM@?$AAN?$AAo?$AA?5?$AAC?$AAo?$AAn?$AAt?$AAr?$AAo?$AAl?$AA?5?$AA?$CI?$AAR?$AAS?$AA2?$AA3?$AA2?$AA?$CJ?$AA?$AA@ 100014d0     ConfigParser.obj
 0001:000004f8       ??_C@_1CO@KJKNEDLA@?$AAL?$AAo?$AAw?$AA?5?$AAE?$AAn?$AAa?$AAb?$AAl?$AAe?$AA?5?$AA?$CI?$AAR?$AAS?$AA4?$AA2?$AA2?$AA?1?$AA4?$AA8?$AA5?$AA?$CJ?$AA?$AA@ 100014f8     ConfigParser.obj
 0001:00000528       ??_C@_1BI@LGOMGNKN@?$AAH?$AAi?$AAg?$AAh?$AA?5?$AAE?$AAn?$AAa?$AAb?$AAl?$AAe?$AA?$AA@ 10001528     ConfigParser.obj
 0001:00000540       ??_C@_19BIEPDBPA@?$AAT?$AAy?$AAp?$AAe?$AA?$AA@ 10001540     ConfigParser.obj
 0001:0000054c       ??_C@_1BK@CENGCIFF@?$AAT?$AAo?$AA_?$AAB?$AAa?$AAu?$AAd?$AA_?$AAR?$AAa?$AAt?$AAe?$AA?$AA@ 1000154c     ConfigParser.obj
 0001:00000568       ??_C@_1BO@CILDMCD@?$AAF?$AAr?$AAo?$AAm?$AA_?$AAB?$AAa?$AAu?$AAd?$AA_?$AAR?$AAa?$AAt?$AAe?$AA?$AA@ 10001568     ConfigParser.obj
 0001:00000588       ??_C@_1CI@IMABDCBP@?$AAL?$AAi?$AAn?$AAe?$AA_?$AAD?$AAr?$AAi?$AAv?$AAe?$AAr?$AA_?$AAC?$AAo?$AAn?$AAt?$AAr?$AAo?$AAl?$AA?$AA@ 10001588     ConfigParser.obj
 0001:000005b0       ??_C@_1BE@GELDBLFK@?$AAT?$AAa?$AAb?$AA_?$AAA?$AAb?$AAo?$AAu?$AAt?$AA?$AA@ 100015b0     ConfigParser.obj
 0001:000005c4       ??_C@_1DA@NCKAKAMN@?$AAT?$AAa?$AAb?$AA_?$AAL?$AAi?$AAn?$AAe?$AA_?$AAD?$AAr?$AAi?$AAv?$AAe?$AAr?$AA_?$AAC?$AAo?$AAn?$AAt?$AAr?$AAo?$AAl?$AA?$AA@ 100015c4     ConfigParser.obj
 0001:000005f4       ??_C@_1CA@LJNFGPHD@?$AAT?$AAa?$AAb?$AA_?$AAF?$AAi?$AAf?$AAo?$AA_?$AAL?$AAe?$AAv?$AAe?$AAl?$AAs?$AA?$AA@ 100015f4     ConfigParser.obj
 0001:00000614       ??_C@_1CK@NLOLPFMM@?$AAT?$AAa?$AAb?$AA_?$AAB?$AAa?$AAu?$AAd?$AAr?$AAa?$AAt?$AAe?$AA_?$AAM?$AAa?$AAp?$AAp?$AAi?$AAn?$AAg?$AA?$AA@ 10001614     ConfigParser.obj
 0001:00000640       ??_C@_1CM@OFMOCLCD@?$AAT?$AAa?$AAb?$AA_?$AAC?$AAr?$AAy?$AAs?$AAt?$AAa?$AAl?$AA_?$AAF?$AAr?$AAe?$AAq?$AAu?$AAe?$AAn?$AAc?$AAy?$AA?$AA@ 10001640     ConfigParser.obj
 0001:0000066c       ??_C@_1CC@FHAFLLA@?$AAB?$AAa?$AAu?$AAd?$AAr?$AAa?$AAt?$AAe?$AA_?$AAM?$AAa?$AAp?$AAp?$AAi?$AAn?$AAg?$AA?$AA@ 1000166c     ConfigParser.obj
 0001:00000690       ??_C@_1DG@MMINKBLM@?$AAF?$AAl?$AAo?$AAw?$AA_?$AAC?$AAo?$AAn?$AAt?$AAr?$AAo?$AAl?$AA_?$AAO?$AAf?$AAf?$AA_?$AAL?$AAe?$AAv?$AAe?$AAl?$AA_?$AAM?$AAa?$AAx?$AA?$AA@ 10001690     ConfigParser.obj
 0001:000006c8       ??_C@_1DG@FFKMCLJC@?$AAF?$AAl?$AAo?$AAw?$AA_?$AAC?$AAo?$AAn?$AAt?$AAr?$AAo?$AAl?$AA_?$AAO?$AAf?$AAf?$AA_?$AAL?$AAe?$AAv?$AAe?$AAl?$AA_?$AAM?$AAi?$AAn?$AA?$AA@ 100016c8     ConfigParser.obj
 0001:00000700       ??_C@_1DE@JAENBBJL@?$AAF?$AAl?$AAo?$AAw?$AA_?$AAC?$AAo?$AAn?$AAt?$AAr?$AAo?$AAl?$AA_?$AAO?$AAn?$AA_?$AAL?$AAe?$AAv?$AAe?$AAl?$AA_?$AAM?$AAa?$AAx?$AA?$AA@ 10001700     ConfigParser.obj
 0001:00000734       ??_C@_1DE@JGMJLLF@?$AAF?$AAl?$AAo?$AAw?$AA_?$AAC?$AAo?$AAn?$AAt?$AAr?$AAo?$AAl?$AA_?$AAO?$AAn?$AA_?$AAL?$AAe?$AAv?$AAe?$AAl?$AA_?$AAM?$AAi?$AAn?$AA?$AA@ 10001734     ConfigParser.obj
 0001:00000768       ??_C@_1DO@FFHHIFI@?$AAR?$AAx?$AA_?$AAI?$AAn?$AAt?$AAe?$AAr?$AAr?$AAu?$AAp?$AAt?$AA_?$AAT?$AAr?$AAi?$AAg?$AAg?$AAe?$AAr?$AA_?$AAL?$AAe?$AAv?$AAe?$AAl?$AA_?$AAM?$AAa?$AAx?$AA?$AA@ 10001768     ConfigParser.obj
 0001:000007a8       ??_C@_1DO@JMHGPCHG@?$AAR?$AAx?$AA_?$AAI?$AAn?$AAt?$AAe?$AAr?$AAr?$AAu?$AAp?$AAt?$AA_?$AAT?$AAr?$AAi?$AAg?$AAg?$AAe?$AAr?$AA_?$AAL?$AAe?$AAv?$AAe?$AAl?$AA_?$AAM?$AAi?$AAn?$AA?$AA@ 100017a8     ConfigParser.obj
 0001:000007e8       ??_C@_1DO@HONDFPK@?$AAT?$AAx?$AA_?$AAI?$AAn?$AAt?$AAe?$AAr?$AAr?$AAu?$AAp?$AAt?$AA_?$AAT?$AAr?$AAi?$AAg?$AAg?$AAe?$AAr?$AA_?$AAL?$AAe?$AAv?$AAe?$AAl?$AA_?$AAM?$AAa?$AAx?$AA?$AA@ 100017e8     ConfigParser.obj
 0001:00000828       ??_C@_1DO@JOMMLPNE@?$AAT?$AAx?$AA_?$AAI?$AAn?$AAt?$AAe?$AAr?$AAr?$AAu?$AAp?$AAt?$AA_?$AAT?$AAr?$AAi?$AAg?$AAg?$AAe?$AAr?$AA_?$AAL?$AAe?$AAv?$AAe?$AAl?$AA_?$AAM?$AAi?$AAn?$AA?$AA@ 10001828     ConfigParser.obj
 0001:00000868       ??_C@_1BO@CLLBHNOO@?$AAF?$AAl?$AAo?$AAw?$AA_?$AAO?$AAf?$AAf?$AA_?$AAL?$AAe?$AAv?$AAe?$AAl?$AA?$AA@ 10001868     ConfigParser.obj
 0001:00000888       ??_C@_1BM@FKEALHLG@?$AAF?$AAl?$AAo?$AAw?$AA_?$AAO?$AAn?$AA_?$AAL?$AAe?$AAv?$AAe?$AAl?$AA?$AA@ 10001888     ConfigParser.obj
 0001:000008a8       ??_C@_1EA@FCDBIJCN@?$AAR?$AAe?$AAc?$AAe?$AAi?$AAv?$AAe?$AA_?$AAI?$AAn?$AAt?$AAe?$AAr?$AAr?$AAu?$AAp?$AAt?$AA_?$AAT?$AAr?$AAi?$AAg?$AAg?$AAe?$AAr?$AA_?$AAL?$AAe?$AAv?$AAe?$AAl?$AA?$AA@ 100018a8     ConfigParser.obj
 0001:000008e8       ??_C@_1EC@JOHHNGND@?$AAT?$AAr?$AAa?$AAn?$AAs?$AAm?$AAi?$AAt?$AA_?$AAI?$AAn?$AAt?$AAe?$AAr?$AAr?$AAu?$AAp?$AAt?$AA_?$AAT?$AAr?$AAi?$AAg?$AAg?$AAe?$AAr?$AA_?$AAL?$AAe?$AAv?$AAe?$AAl@ 100018e8     ConfigParser.obj
 0001:0000092c       ??_C@_1BI@LMBHJBLG@?$AAT?$AAa?$AAb?$AA_?$AAO?$AAp?$AAt?$AAi?$AAo?$AAn?$AAs?$AA?$AA@ 1000192c     ConfigParser.obj
 0001:00000944       ??_C@_1BI@GEBICGMH@?$AAF?$AAi?$AAf?$AAo?$AA_?$AAL?$AAe?$AAv?$AAe?$AAl?$AAs?$AA?$AA@ 10001944     ConfigParser.obj
 0001:0000095c       ??_C@_1M@MNHBCACD@?$AAT?$AAi?$AAt?$AAl?$AAe?$AA?$AA@ 1000195c     ConfigParser.obj
 0001:00000968       ??_C@_1CE@FHCKENKN@?$AAC?$AAr?$AAy?$AAs?$AAt?$AAa?$AAl?$AA_?$AAF?$AAr?$AAe?$AAq?$AAu?$AAe?$AAn?$AAc?$AAy?$AA?$AA@ 10001968     ConfigParser.obj
 0001:0000098c       ??_C@_1CE@EOJPOKCA@?$AAA?$AAp?$AAp?$AAl?$AAi?$AAc?$AAa?$AAt?$AAi?$AAo?$AAn?$AA_?$AAT?$AAi?$AAt?$AAl?$AAe?$AA?$AA@ 1000198c     ConfigParser.obj
 0001:000009b0       ??_C@_15JJPIMNBO@?$AAr?$AAb?$AA?$AA@ 100019b0     ConfigParser.obj
 0001:000009b8       ??_C@_1BI@MHELFDAB@?$AA?2?$AAW?$AAi?$AAn?$AAd?$AAo?$AAw?$AAs?$AA?2?$AA?$CF?$AAs?$AA?$AA@ 100019b8     ConfigParser.obj
 0001:000009f8       _KLibFreeShareMem          100019f8 f i buspcie950.obj
 0001:00000a16       ?DllEntry@@YAHPAUHINSTANCE__@@KPAX@Z 10001a16 f   buspcie950.obj
 0001:00000aab       ?GetBrandingData@@YAHPAU_CONFIG_DATA_@@PAG@Z 10001aab f   buspcie950.obj
 0001:00000ac3       ?Deinit@@YAXPAX@Z          10001ac3 f   buspcie950.obj
 0001:00000cb7       ?Init@@YAPAXPBG@Z          10001cb7 f   buspcie950.obj
 0001:00001e15       __tfsubstring              10002e15 f   ConfigParser.obj
 0001:00001e50       ?_ffeosubsec@@YAHPAXQAG@Z  10002e50 f   ConfigParser.obj
 0001:00001eaf       _InitializeConfigInfo      10002eaf f   ConfigParser.obj
 0001:00001ef8       ?ValidateCrystalFrequency@@YAHH@Z 10002ef8 f   ConfigParser.obj
 0001:00001fa4       ?ValidateValues@@YAXPAU_CONFIG_DATA_@@@Z 10002fa4 f   ConfigParser.obj
 0001:000020d2       ?_textractValue@@YAPAGPAG@Z 100030d2 f   ConfigParser.obj
 0001:00002104       _ParseConfigFile           10003104 f   ConfigParser.obj
 0001:00002dcc       _BusTransBusAddrToStatic   10003dcc f   ceddk:CEDDK.dll
 0001:00002dd2       _BusTransBusAddrToVirtual  10003dd2 f   ceddk:CEDDK.dll
 0001:00002dd8       _CreateBusAccessHandle     10003dd8 f   ceddk:CEDDK.dll
 0001:00002dde       _EventModify               10003dde f   coredll:COREDLL.dll
 0001:00002de4       _KernelLibIoControl        10003de4 f   coredll:COREDLL.dll
 0001:00002dea       _InterruptDone             10003dea f   coredll:COREDLL.dll
 0001:00002df0       _DeactivateDevice          10003df0 f   coredll:COREDLL.dll
 0001:00002df6       _GetDeviceInformationByDeviceHandle 10003df6 f   coredll:COREDLL.dll
 0001:00002dfc       _ActivateDeviceEx          10003dfc f   coredll:COREDLL.dll
 0001:00002e02       _wsprintfW                 10003e02 f   coredll:COREDLL.dll
 0001:00002e08       _CreateThread              10003e08 f   coredll:COREDLL.dll
 0001:00002e0e       _InterruptInitialize       10003e0e f   coredll:COREDLL.dll
 0001:00002e14       _LoadIntChainHandler       10003e14 f   coredll:COREDLL.dll
 0001:00002e1a       @__security_check_cookie@4 10003e1a f   corelib0:x86secgs.obj
 0001:00002e40       _wcstoul                   10003e40 f   corelib1:COREDLL.dll
 0001:00002e46       _free                      10003e46 f   corelib1:COREDLL.dll
 0001:00002e4c       _malloc                    10003e4c f   corelib1:COREDLL.dll
 0001:00002e52       _wcstol                    10003e52 f   corelib1:COREDLL.dll
 0001:00002e58       __chkstk                   10003e58 f   corelib1:COREDLL.dll
 0001:00002e5e       _wcschr                    10003e5e f   corelib1:COREDLL.dll
 0001:00002e64       _wcsrchr                   10003e64 f   corelib1:COREDLL.dll
 0001:00002e6a       _fgetws                    10003e6a f   corelib1:COREDLL.dll
 0001:00002e70       _fclose                    10003e70 f   corelib1:COREDLL.dll
 0001:00002e76       __wtol                     10003e76 f   corelib1:COREDLL.dll
 0001:00002e7c       _feof                      10003e7c f   corelib1:COREDLL.dll
 0001:00002e82       __wfopen                   10003e82 f   corelib1:COREDLL.dll
 0001:00002e88       _swprintf                  10003e88 f   corelib1:COREDLL.dll
 0001:00002e8e       ___report_gsfailure        10003e8e f   corelib1:COREDLL.dll
 0001:00002e94       __IMPORT_DESCRIPTOR_CEDDK  10003e94     ceddk:CEDDK.dll
 0001:00002ea8       __IMPORT_DESCRIPTOR_COREDLL 10003ea8     coredll:COREDLL.dll
 0001:00002ebc       __NULL_IMPORT_DESCRIPTOR   10003ebc     ceddk:CEDDK.dll
 0002:00000000       __imp__BusTransBusAddrToVirtual 10004000     ceddk:CEDDK.dll
 0002:00000004       __imp__CreateBusAccessHandle 10004004     ceddk:CEDDK.dll
 0002:00000008       __imp__BusTransBusAddrToStatic 10004008     ceddk:CEDDK.dll
 0002:0000000c       \177CEDDK_NULL_THUNK_DATA  1000400c     ceddk:CEDDK.dll
 0002:00000010       __imp__EventModify         10004010     coredll:COREDLL.dll
 0002:00000014       __imp__KernelLibIoControl  10004014     coredll:COREDLL.dll
 0002:00000018       __imp__DisableThreadLibraryCalls 10004018     coredll:COREDLL.dll
 0002:0000001c       __imp__InterruptDone       1000401c     coredll:COREDLL.dll
 0002:00000020       __imp__WaitForSingleObject 10004020     coredll:COREDLL.dll
 0002:00000024       __imp__CloseHandle         10004024     coredll:COREDLL.dll
 0002:00000028       __imp__DeactivateDevice    10004028     coredll:COREDLL.dll
 0002:0000002c       __imp__RegQueryValueExW    1000402c     coredll:COREDLL.dll
 0002:00000030       __imp__RegSetValueExW      10004030     coredll:COREDLL.dll
 0002:00000034       __imp__GetDeviceInformationByDeviceHandle 10004034     coredll:COREDLL.dll
 0002:00000038       __imp__ActivateDeviceEx    10004038     coredll:COREDLL.dll
 0002:0000003c       __imp__RegCreateKeyExW     1000403c     coredll:COREDLL.dll
 0002:00000040       __imp__wsprintfW           10004040     coredll:COREDLL.dll
 0002:00000044       __imp__CreateThread        10004044     coredll:COREDLL.dll
 0002:00000048       __imp__InterruptInitialize 10004048     coredll:COREDLL.dll
 0002:0000004c       __imp__CreateEventW        1000404c     coredll:COREDLL.dll
 0002:00000050       __imp__LoadIntChainHandler 10004050     coredll:COREDLL.dll
 0002:00000054       __imp__RegCloseKey         10004054     coredll:COREDLL.dll
 0002:00000058       __imp__RegOpenKeyExW       10004058     coredll:COREDLL.dll
 0002:0000005c       __imp__wcstoul             1000405c     corelib1:COREDLL.dll
 0002:00000060       __imp__free                10004060     corelib1:COREDLL.dll
 0002:00000064       __imp__malloc              10004064     corelib1:COREDLL.dll
 0002:00000068       __imp__wcstol              10004068     corelib1:COREDLL.dll
 0002:0000006c       __imp___chkstk             1000406c     corelib1:COREDLL.dll
 0002:00000070       __imp__wcschr              10004070     corelib1:COREDLL.dll
 0002:00000074       __imp__wcsrchr             10004074     corelib1:COREDLL.dll
 0002:00000078       __imp__fgetws              10004078     corelib1:COREDLL.dll
 0002:0000007c       __imp__fclose              1000407c     corelib1:COREDLL.dll
 0002:00000080       __imp___wtol               10004080     corelib1:COREDLL.dll
 0002:00000084       __imp__feof                10004084     corelib1:COREDLL.dll
 0002:00000088       __imp___wfopen             10004088     corelib1:COREDLL.dll
 0002:0000008c       __imp__swprintf            1000408c     corelib1:COREDLL.dll
 0002:00000090       __imp____report_gsfailure  10004090     corelib1:COREDLL.dll
 0002:00000094       \177COREDLL_NULL_THUNK_DATA 10004094     coredll:COREDLL.dll
 0002:00000098       ?dpCurSettings@@3U_DBGPARAM@@A 10004098     buspcie950.obj
 0002:000004dc       ___security_cookie         100044dc     corelib0:seccinit.obj
 0002:000004e0       ___security_cookie_complement 100044e0     corelib0:seccinit.obj
 0002:000004e8       ?Pcie950BusInfo@@3UPCIE950_BUS_INFO@@A 100044e8     buspcie950.obj
 0002:00000588       ?m_pDispatchThread@@3PAXA  10004588     buspcie950.obj

 entry point at        0000:00000000

 Static symbols

 0001:00000a2e       ?BusIstThread@@YAKPAX@Z    10001a2e f   buspcie950.obj
 0001:00000b46       ?ReadKeyList@@YAHPAUHKEY__@@PBGKPAK2@Z 10001b46 f   buspcie950.obj
 0001:00000c1c       ?ReadKeyDword@@YAHPAUHKEY__@@PBGPAK@Z 10001c1c f   buspcie950.obj
 0001:00000c5b       ?WriteKeyDword@@YAHPAUHKEY__@@PBGK@Z 10001c5b f   buspcie950.obj
 0001:00000c7e       ?WriteKeyString@@YAHPAUHKEY__@@PBG1@Z 10001c7e f   buspcie950.obj
